:020000020000FC
:1000000084C0FFB6989B39C01123B9F4B29B29C0B4
:020010000BC023
:10001600FFB6112713BF89B3807F9D998F608BBB75
:1000260037C0962CA72CB82C662477248824CC2499
:10003600DD24EE24B29B07C0139590E093BF9EEC9F
:1000460092BF93E093BF123058F061F0143018F06D
:1000560029F49B2D08C09091690005C0992703C01B
:10006600992D01C09A2DB29992959F7089B3807F80
:10007600982B0BC09D9912C0112799B3907FB29B04
:1000860003C08FEF9F6002C09229812D9BBB88BB66
:1000960092E0B29B93E095BFFFBE1895112341F401
:1000A600B29B29C090E093BF98E392BF93E093BFC1
:1000B600B2991395133038F089F0B29B1CC099B3EE
:1000C600907F9F6006C0B29B17C099B3907F92291C
:1000D600967F812D859585958370D8CFB29B03C079
:1000E60099B3907FF6CF99B3907F812D82958F70CB
:1000F600982B83E0CBCF112799B3907F9229812D3E
:100106008370C4CF21E02EBF2FE52DBF2FEF2ABB72
:100116002BE027BB20E42BBF21E029BFE4D362E01C
:10012600B0D298D2F89463E0ACD22FEF28BB2BBBA9
:1001360091D2112713BB10936800E2D380F360E0DD
:1001460061F99FD2989400FDE1D001FDF8D002FD3F
:1001560051D104FDE2D005FD00D109F7202F2295EB
:10016600022B66247724882455243324442413D070
:1001760093E095BF789475D2889400FD3AD040F00C
:1001860001FD47D028F002FD24D010F004D0F2CFB4
:100196002E3081F7C7CF98990DC0242D6FEF2627F3
:1001A6002F70222E112349F469B3607F262BB29B50
:1001B6002BBB03C06C2C7D2C8E2C232D25296FEF99
:1001C6002627122E112321F4B29968BBB29B18BAC6
:1001D600089520916E002A9519F020936E000895D7
:1001E60020917E0020936E00C6D2C8F3C1F3E0D101
:1001F60021C020916E002A9519F020936E00089573
:1002060020916C0020936E00B6D2C8F3C1F39DD145
:1002160011C020916F002A9519F020936F00089560
:1002260020916D0020936F00A1D2C8F3C1F32093F3
:10023600790003D0989488940895989AB0E0AFE82E
:1002460022E099992D91233008F008952D91662783
:1002560020FD626021FD6160562E2695269520615F
:100266003AD02093690020917900263030F09B998E
:100276002D919C9911C09A9918C0CD90DD902D9121
:10028600219529D0E22E2C2D219525D0C22E2D2D5B
:10029600219521D0D22E08956D912D9129D0C62E6B
:1002A6006D912D9125D0D62EEACF6D912C912F7080
:1002B60023FD206F1DD0C62E6D9162956F705C91E7
:1002C6005295507F652B2D9122952F7023FD206F1F
:1002D6000FD0D62ED4CF222351F0622F2A7A60FD7A
:1002E600246062FD216064FD206466FD206108953E
:1002F60027FD06C0222311F467FF08956FE70895CE
:100306002F3F11F467FD089560E808953091750058
:1003160020917C0050917E0006C03091760020919D
:100326007D0050917F003093770020936A005093B0
:100336006C0050936E0020E005D11894089520912A
:100346007C0020936B0020917E0020936D0020930B
:100356006F00609180002FD20DC020917D00209308
:100366006B0020917F0020936D0020936F006091B9
:1003760081001ED209F0089550917400A0E9B0E002
:10038600552309F15A952D91203CE9F0253821F4A1
:10039600999A5A952D91F4CF253931F45A952D9184
:1003A600203171F79B9AECCF253739F45A952D9168
:1003B600203131F02C3031F0E3CF06D009F3089527
:1003C6009C9A08959A9A0895237081F02A9559F077
:1003D6002A9531F05A9561F02D915A9549F02D9153
:1003E6005A9531F02D915A9519F02D91189408953A
:1003F6009894089520917C0020936A0020917E00B5
:1004060020936C0020936E0060918000D4D139F067
:1004160051E008C0209175002093770008950FD011
:10042600C9F352E063E02DD115D161E02AD112D192
:1004360063E027D10FD15A95C1F798940895E2E168
:10044600F5E06AD029F0E8E1F5E066D009F0089514
:1004560033273093820030938300309384005A957B
:100466002D91253831F433955A952D912093850099
:10047600F6CF213A21F45A952D91223011F0989415
:1004860008955A952D912537D1F75A952D912830F3
:10049600B1F75A952D91253719F1253911F40CD05C
:1004A600F8CF293011F40BD0F4CF213811F411D044
:1004B600F0CF8ADF71F308955A950D9008955A95F5
:1004C6002D910A943395203309F0089530938200D4
:1004D60008955A952D91213009F00895300D08950B
:1004E6005A952D91213019F0243059F008955A95D6
:1004F6002D91253909F008955A952D91243009F04A
:1005060001C03068309383001894089505010904EA
:10051600A10105010905A10150917400A0E9B0E00F
:1005260036E005902D91201519F45A953A95C9F79C
:10053600089560918900693309F0089562E0209179
:100546006800262720936800D3C0F3DFB0E0A7E851
:1005560060E02C912F7009F062E02D91207F09F068
:1005660061E0362E2D913327662708D0622BAF38EF
:10057600E0F3462E232D232B322E08955D9122275C
:10058600583591F05A3291F05C3271F028E05F54A0
:1005960051F021E05A9539F022E05A9521F024E0F5
:1005A6005A9509F02227089532600895316008951A
:1005B600209182002A95B0E0A7E8A20F66272D9128
:1005C600203009F461602F3F09F468602D912030D6
:1005D60009F464602F3F09F46260462E209183007F
:1005E600622F6F77A7E8A60F6D915C9127FF08C071
:1005F6005695679556956795569567955695679559
:100606009E9906C0262F252B09F151FD9D9A9E9A8B
:100616009D990BC0562F52956795652B222761FD34
:10062600226060FD2160322E0895222765FD21603B
:1006360062FD226051FD246061FD286060FD20613D
:1006460063FD206264FD206450FD2068322E08950B
:1006560039E101C032E303D03A95E9F7089544E65B
:1006660001C04AE003D04A95E9F7089524E6000060
:1006760000000000000000002A95C9F7089523E055
:10068600F6CF78EA7260DF987FB920D06FB91ED0B6
:10069600DF9A08957260DF987FB918D02D9115D032
:1006A6005A95E1F7DF9A0895DF987FB90FD0222790
:1006B60015D0DF9A0895DF987FB908D022270ED08B
:1006C6002D935A95D9F7DF9A08952FB920E42EB9BC
:1006D6003BE13DB92EB126FFFCCF08952FB920E4AA
:1006E6002EB93BE13DB92EB126FFFCCF2FB10895BF
:1006F600FAE0EEE561E08BD170E258E0CBDF60E432
:1007060078EEC0DF20E120937000B4D009F00895A0
:1007160060E878EEB7DF22272093710020937200FD
:1007260003C060E078E3AEDF6091680070E1AADFA5
:1007360061E078E3A7DF20E220937000C6D009F4D9
:100746000895243041F4209171002395209371007F
:10075600283C39F709C02E3039F4209172002395D0
:10076600209372002530E9F622230895AFE8B0E021
:1007760020916B0004C0A7E8B0E020916A002093A6
:100786007000A3D029F0243011F00894089508953C
:1007960070E38ADF522F2F9378E086DF2D935A95E8
:1007A600D9F778EC64E06EDF2F91222388940895C0
:1007B600FAE0EEE709C0FAE0E6E706C0FAE0EEE6A0
:1007C60003C062E1FAE0E6E622D170E258E062DFB9
:1007D60020E1209370004ED009F0089578EE60E293
:1007E60060937A004FDF2E912E9106D021F420EAF5
:1007F600209370003FC00895A0E9B0E020937800F0
:1008060022272093740020E02093700033D009F053
:10081600089570E349DF20937300522F78E044DF98
:100826002D935A95D9F778EC64E02CDF209174006B
:1008360050917300250F2093740020917700521772
:1008460030F020917400509178002517E0F218944A
:100856000895FAE0E6E5DAD0A0E6B0E070E258E006
:1008660019DF20E12093700005D009F0089520E8F3
:10087600209370002227209371002093720025D0C8
:1008860009F40895243041F42091710023952093B2
:100896007100283CA1F709C02E3039F4209172006E
:1008A600239520937200253051F7263061F460912C
:1008B6007A00603111F060E101C060E260937A0075
:1008C60078EEE0DEE1F6222308956091700070EF85
:1008D600D9DE78ECE9DE2078E1F360E8D3DE78EF64
:1008E600E3DE2F70089578E864E1CCDE78E760E215
:1008F600C9DE60E0C7DE78E6D7DE2170E9F3089549
:100906003DD0D0F158EC90D054D0B1F55ADFA1F5D6
:1009160068E054DF89F56091920050DF30919400D1
:10092600E9E9F0E00781002309F404E02089209337
:10093600800024892F7020937C00268920937500DF
:10094600208D20937E003130A1F0043091F0E2EB4F
:10095600F0E027812295022B2089209381002489AB
:100966002F7020937D00268920937600208D20937A
:100976007F006FDF889408950894089578ED61EC00
:1009860081DE78EC60E27EDE78EE64E07BDE78EF96
:100996008BDE207C61F078ED203821F06BEC72DE86
:1009A600689403C069EC6EDEE89488940895089410
:1009B600089528E02093770078EE61E063DE78EE14
:1009C60073DE2170E1F758EC2FD060E070EE5ADE4E
:1009D60068E0F8DE09F008952091970020937700EB
:1009E60078EE61E04FDE78EE5FDE2170E1F758ECDD
:1009F6001BD0FAE0E6E42FDF09F008955EE114D09B
:100A060061E070EE3FDEFAE0EEE425CF662767FD93
:100A160060E807D058E025912D935A95E1F75E934B
:100A26006E93B0E0A0E6089578EC60E42BDE78ECF7
:100A36003BDE2074E1F360E425DE5A95C1F70895A4
:100A46000005010000000000000901000000000090
:100A5600210A000000000000210900020000010038
:100A660080060001000012008006000200008000DF
:100A7600810600220000800081060022010080001D
:100FC0004D535848494431207665722E332E3320D4
:100FD0002020202032342E30312E323032320D0A91
:100FE000415454696E7934342F3834202020202025
:100FF000202020202020286329206361726F0D0AA1
:00000001FF
